:100000000C9441030C9479030C9479030C947903B8
:100010000C9479030C9479030C9479030C94790370
:100020000C9479030C9479030C9433110C946F1095
:100030000C94421F0C9479030C9479030C9479036B
:100040000C9479030C9479030C9479030C94790340
:100050000C9479030C94011F0C9479030C9479038C
:100060000C9479030C9479030C9479030C94790320
:100070000C9479030C9479030C9479030C94790310
:100080000C941C230C9479030C9479030C9479033D
:100090000C9479030C9479030C9479030C947903F0
:1000A0000C9479030C9479030C947903E209E20926
:1000B000140A140A890A310C310C310CA50A830B7D
:1000C000940B940B860EAD0E5110AD0E5110F90E1F
:1000D0001C0F511012102110362539253F255225AD
:1000E0002D2604276C269926CA2607634236B79B1D
:1000F000D8A71A39685618AEBAAB558C1D3CB7CC88
:100100005763BD6DEDFD753EF6177231BF000000FF
:10011000803F08000000BE922449123EABAAAA2AE2
:10012000BECDCCCC4C3E00000080BEABAAAAAA3EFD
:1001300000000000BF000000803F00000000000839
:100140004178D3BB4387D1133D190E3CC3BD4282D6
:10015000AD2B3E68EC8276BED98FE1A93E4C80EF94
:10016000FFBE01C4FF7F3F00000000006261636BBF
:100170006C696768742064656372656173653A20B1
:1001800025750A006261636B6C6967687420696E2B
:100190006372656173653A2025750A006261636B5D
:1001A0006C696768742064697361626C650A0062D7
:1001B00061636B6C6967687420656E61626C650A67
:1001C000006261636B6C6967687420746F67676C49
:1001D000653A2025750A0044454255473A2064692E
:1001E0007361626C65642E0A0044454255473A20AB
:1001F000656E61626C65642E0A000631FF0974A1A8
:10020000010975150026FF00952075088102097601
:10021000150026FF00952075089102C00501098090
:10022000A101850319012AB700150126B700950120
:1002300075108100C0050C0901A101850419012A6E
:10024000A002150126A002950175108100C00501CC
:100250000906A101050719E029E715002501950800
:10026000750181029501750881010507190029FFB3
:10027000150026FF0095067508810005081901295B
:1002800005950575019102950175039101C05B43C8
:100290005D005B445D005B535D005B575D005B523E
:1002A0005D0009025B00030100A0FA0904000001DF
:1002B000030101000921110100012240000705810D
:1002C00003080001090401000103000000092111D5
:1002D0000100012232000705820320000109040207
:1002E0000002030000000921110100012222000781
:1002F000058303200001070503032000011201000C
:100300000200000008A803F36702000102000110C8
:10031000035000720065006F006E0069006300000A
:10032000000A034F004C004B004200000004030988
:100330000435001E001F002000210022002300249D
:10034000002500260027002A002B0014001A0008B0
:1003500000150017001C0018000C00120013004CC0
:1003600000290004001600070009000A000B000D18
:10037000000E000F0033003400E1001D001B0006DA
:100380000019000500110010003600370038002861
:1003900000AC5DE000E200E300AA5D2C002C00ABA5
:1003A0005D5000510052004F0035001E001F00201C
:1003B0000021002200230024002500260027002A17
:1003C000002B0014001A00090013000A000D000F92
:1003D0000018001C0033004C002900040015001612
:1003E00000170007000B00110008000C0012003479
:1003F00000E1001D001B000600190005000E0010A2
:10040000003600370038002800AC5DE000E200E371
:1004100000AA5D2C002C00AB5D5000510052004F33
:100420000035001E001F00200021002200230024B0
:10043000002500260027002A002B00340036003754
:100440000013001C0009000A00060015000F004CF4
:1004500000290004001200080018000C0007000B1F
:10046000001700110016003800E100330014000DE1
:10047000000E001B00050010001A0019001D0028C6
:1004800000AC5DE000E200E300AA5D2C002C00ABB4
:100490005D5000510052004F0035021E021F022025
:1004A0000221022202230224022502260227022A16
:1004B0000035021E021F0220022102220223022412
:1004C000022502260227024C004C003A003B003C69
:1004D000003D003E003F002D022E022F023002316F
:1004E0000201004000410042004300440045003248
:1004F0000264024A004D00010001000100010001F8
:10050000000100010001000100AB00AA00A900AE3B
:100510000035001E001F00200021002200230024BF
:10052000002500260027002A0035001E001F00209D
:100530000021002200230024002500260027004C73
:10054000004C003A003B003C003D003E003F002DC7
:10055000002E002F00300031000100400041004219
:1005600000430044004500320064004B004E00018F
:100570000001000100010001000100010001000173
:1005800000AB00AA00A900AE003A003B003C003DD1
:10059000003E003F0040004100420043004400454F
:1005A000000100005C015C0100010001000100008D
:1005B000000000010001004C0001000100295C1D49
:1005C0005C1E5C135C0A5CA75DA85DA95D0100016F
:1005D0000001002B5C2A5C265C275C2C5C2D5C01F6
:1005E0000001000100010001000100010001000103
:1005F00000010001000100010001000100010001F3
:10060000004F6E6573686F743A2061637469766534
:100610003A2025640A000A002530325820006B6514
:1006200079626F6172645F7265706F72743A2000F4
:100630005B735D000A002530313662003A200025E8
:10064000303258000A722F6320303132333435365D
:100650003738394142434445460A000A00253032C2
:1006600058006C65645F7461736B3A20006261636B
:100670006B6C6967687420737465703A2025750A1D
:10068000000011241FBECFEFDAE0DEBFCDBF04B6FD
:1006900003FE18C080911C0790911D07A0911E07B2
:1006A000B0911F078730904BA740B04B59F4109280
:1006B0001C0710921D0710921E0710921F07E0E002
:1006C000F8E3099515E0A0E0B1E0EEEBFCE502C02F
:1006D00005900D92A23DB107D9F727E0A2EDB5E054
:1006E00001C01D92AC31B207E1F70E94BF1B0C9410
:1006F0005D2E0C940000FF93EF93E091D205F091F2
:10070000D305309709F00995EF91FF910895FC0109
:100710008591803011F0EFDFFBCF0895FF27E0E2F5
:1007200030E247FF0CC0419597FF09C0EDE26095AC
:10073000709580959095611D711D811D911D27FFFC
:1007400002C0219530E350E2AA27660F771F881F69
:10075000991FAA1FA41710F0A41B63955A95A9F717
:10076000AA3008F0A95FA05DAF93F39561157105FC
:100770008105910541F7ED3211F4EF93F395F217EE
:1007800018F43F93F395FBCF8F91B5DFFA95E1F71E
:100790000895E991F9918591803021F0853219F021
:1007A000AADFF9CF089520E0E89455915532C1F3BE
:1007B000503311F4689455915A3348F4505390F3E0
:1007C000220F022E220F220F200D250FF4CF0EF440
:1007D000219589919991533619F3533729F153355E
:1007E00059F1BC0188279927E8945C3621F4899156
:1007F000999168945591543639F446EF7EF077FF1D
:100800000DC08FEF9FEF0AC055374AE039F05835D9
:1008100040E121F0523642E009F00895FF93EF9352
:100820007DDFEF91FF91B7CFFF93EF93FC018191B3
:100830008030B9F360DFFBCFFF93EF9368DFF1CF38
:10084000DF93CF93CDB7DEB72596A3DFCF91DF91AE
:1008500008958F929F92AF92BF92CF92DF92EF92C4
:10086000FF920F931F93CF93DF93CDB7DEB7AD9772
:100870000FB6F894DEBF0FBECDBFFC010081D18062
:1008800083819481892B39F01FEFD11206C091E04A
:100890000F3F19F403C091E001C090E090FF02C047
:1008A0000C94700C7F0185E0DE01999601900D9209
:1008B0008A95E1F7D70112962C9189A59AA5222352
:1008C00049F00E949D12182F682F89A59AA50E94B1
:1008D000FF1403C00E94D314182FBCE31B9FF00128
:1008E00011241CE0D19EE00DF11D1124E00FF11D3B
:1008F000EE0FFF1FEF5CFC4F05911491D70112968C
:100900009C91093ABDE51B0701F148F4073AFDE562
:100910001F0779F0083A2DE5120781F035C00B3A30
:100920003DE51307C9F0B0F00C3A8DE51807F9F072
:100930002BC0992309F4C0C480E004C0992309F4B2
:10094000BBC481E00E94CA28B7C4992309F4B4C487
:1009500082E0F8CF83E001C084E0911105C00E94DD
:1009600034150E94D924A8C40E945915FACF85EEE7
:10097000992331F00E94F7150E940D2176989CC4AE
:100980000E94A015769A98C40D312CE5120731F417
:10099000992309F426C10E94421B8EC40E31ACE596
:1009A0001A0731F4992309F41CC10E94281B84C43E
:1009B0000F31BCE51B0741F4992309F412C1809162
:1009C000D10680FDF2CFE7CF0A32ECE51E0741F4F5
:1009D000992309F406C18091D40690E001960BC0DA
:1009E0000B32FCE51F07A1F4992309F4FAC08091AA
:1009F000D40690E0089669E070E00E94362E80935D
:100A0000D40664E070E084E091E00E94682754C45A
:100A1000992309F4E6C00E3B2CE51207C9F188F4CE
:100A20000C3B5CE51507E1F00D3B8CE5180709F080
:100A3000D8C08091B00687708E7F8093B00680E02A
:100A400020C0003CACE51A0709F47DC008F449C099
:100A5000013CECE51E0709F0C4C00E940D212CC426
:100A60008091B006877088618093B006887F91E09E
:100A700009F490E08091B00690FB80F98093B00675
:100A800083E00E9455208091B0060E94082114C482
:100A90008091B006982F969596959695A1F0915EC7
:100AA000990F990F990F8770892B8093B006887FD3
:100AB00091E009F490E08091B00690FB80F980937A
:100AC000B0060E9408218091AF0680FF84C080910B
:100AD000B0068695869586951F928F938CE691E059
:100AE00029C02091B006822F869586958695482F3D
:100AF00050E04330510554F48F5F982F990F990FB0
:100B0000990F822F8770892B8093B0068091B00651
:100B100081608093B0060E9408218091AF0680FF1B
:100B20005AC08091B0068695869586951F928F93C0
:100B300084E891E09F938F930E9420040F900F9080
:100B40000F900F9048C01091B00611708091AF06C1
:100B500080FF0CC01F921F9381EC91E09F938F93B5
:100B60000E9420040F900F900F900F908091B0067C
:100B70001123B9F080FFA0C38E7F8093B0060E943E
:100B800008218091AF0680FF08C08CE991E09F9317
:100B90008F930E9420040F900F9080E00E945520B8
:100BA0008BC380FD89C381608093B006813019F4C6
:100BB00089E08093B0068091B0060E940821809160
:100BC000AF0680FF08C08FEA91E09F938F930E9449
:100BD00020040F900F908091B0068695869586959B
:100BE000DDCF06323CE5130731F4992309F456C0F2
:100BF0000E94822161C30732FCE51F0731F499236B
:100C000009F44CC00E94122357C308322CE5120786
:100C100041F4992309F442C08091AD068111F2CFCD
:100C2000E7CF0C323CE5130729F49923B9F10E9470
:100C3000792142C30D325CE5150749F4992371F11E
:100C40001092AE0668E070E084E291E0DECE0E32F3
:100C50008CE5180739F4992309F18091AE068111CA
:100C6000EFCFE5CF0932ACE51A07C1F49923B1F013
:100C70000E940C232091040230E02F5F3F4F23702D
:100C800033272093040248E2429FC001439F900D06
:100C9000112465E070E08C599E4FB7CE4091AD06AF
:100CA000411105C08091AE06882309F431C2992311
:100CB00009F44BC0003E110561F40E940C2381E051
:100CC0008093D5051092D4051092A20610929E062C
:100CD000F3C2023E110571F40E940C238091D505E8
:100CE000882319F081E08093D4051092D5051092E5
:100CF000A206E2C2033E110591F48091D405882337
:100D000021F10E940C231092D50581E08093A20668
:100D100010929F061092A1061092A006CDC2023535
:100D2000110531F480918A0290918B020A9708C0D4
:100D30000135110551F480918A0290918B020A9637
:100D400090938B0280938A02B7C280910402811132
:100D50000BC0F701818125E030E0281B310980813B
:100D6000805FD82EFCE01DC0813079F4D701119648
:100D70008C91119725E030E0281B3109D22EDD0C33
:100D8000DD0CD20E8C918D5C2EC0823071F4F70197
:100D9000818125E030E0281B310980818D5CD82ECF
:100DA000F7E02F9FD00C112422C08330F1F483E2AE
:100DB000EEE0F5E0DE01119601900D928A95E1F7E3
:100DC000D7018C91FE01E80FF11D11968C9125E061
:100DD00030E0281B3109D0848D2DBCE02B9F800D85
:100DE000112469E0D62ED80E02C05CE0D52E9923DE
:100DF000A1F0442319F08D2D0E94B91B8091D505D7
:100E0000882391F080919E06E82FF0E0E257F94F99
:100E1000D0828F5F80939E0607C0442329F08D2DDA
:100E20000E949A1B0E946A220115110509F044C212
:100E3000F7018281882309F4D0C11092B3060430EF
:100E4000FDE51F0758F40B3F2CE5120780F4C8019D
:100E500082509C45449708F0AAC109C002363DE57E
:100E6000130729F0063A5DE5150709F0A0C10E94B5
:100E70006319909379068093780601318CE5180701
:100E800009F4CEC008F045C00930ACE51A0709F4F2
:100E9000A5C000F50530ECE51E0709F48DC078F417
:100EA00003302CE5120709F47FC008F081C002303E
:100EB0001C4509F01DC180917806816017C107307B
:100EC0008CE5180709F482C008F084C08091780688
:100ED00080610CC10D30ACE51A0709F48DC070F4C7
:100EE0000B30ECE51E0709F47FC008F081C080914B
:100EF00078068860846080937806B3C00F302CE554
:100F0000120709F485C008F087C080917806877FB2
:100F1000EDC00E3F5CE5150709F476C008F5053114
:100F20009CE5190709F48EC068F40331BCE51B0782
:100F300009F47AC008F0B8C00E9484158091780640
:100F40008F77D4C00C3FFCE51F07D1F108F058C0E3
:100F50000B3F1C4509F0CCC080917906816033C0FD
:100F600002305DE5150709F4ABC070F401159DE58D
:100F7000190709F460C008F07EC08091790682608C
:100F800081608093790684C00236BDE51B0709F4B1
:100F90009DC0063AEDE51E0709F4A2C003301D45C9
:100FA00009F0A6C060E08DC08091780682609EC086
:100FB0008091780684609AC080917806886096C097
:100FC0008091790682608093790692C0809178063C
:100FD00080628CC080917806806488C00E948415ED
:100FE00080917806806882C0809178068E7F7EC06E
:100FF000809178068D7F7AC0809178068B7F76C04D
:10100000809179068E7FDFCF809179068D7FDBCF4F
:10101000809178068F7E6AC0809178068F7D66C049
:10102000809178068F7B62C080917806877F8B7F66
:10103000809378061BC0809179068D7F8E7F809388
:1010400079062BC08091780682FB222720F991E057
:10105000922790FB82F990FB83F98093780699237D
:1010600029F064E070E085E492E01BC062E070E08B
:1010700085E192E016C080917906982F9095917045
:101080008E7F892B90FB81F980937906992329F033
:1010900064E070E085E292E004C062E070E085E028
:1010A00092E00E94682724C00E94841580917806EF
:1010B00087FB222720F991E0922790FB87F916C041
:1010C00061E08EE090E00E945D2912C08091780678
:1010D00084FB222720F991E0922790FB84F906C037
:1010E00080917806982F909590FB80F980937806F0
:1010F000609178061091790684E090E00E945D2965
:10110000612F82E290E00E945D290E948415D4C084
:10111000043F5CE51507A1F406E221EE40EE64EF22
:101120007CE50AC0083DBCE51B0709F081CE06E25C
:1011300021EE41EE68ED7CE5C7010E94CA1FBCC0EC
:10114000053F8CE51807A0F4093D9CE5190731F42B
:1011500007E225EE45EE69ED7CE5EECF0A3DACE514
:101160001A0701F708E221E045EE6AED7CE5E4CFDD
:10117000063FECE51E0731F406E221EE42EE66EF93
:101180007CE5DACF063FFCE51F0730F407E225EEE9
:1011900044EE65EF7CE5D0CF073F2CE5120709F060
:1011A00047CE07E225EE46EE67EF7CE5C5CF063178
:1011B0003CE5130719F5809163068A7A91E009F4FA
:1011C00090E09093D605882311F065E301C069E2B1
:1011D00089E196E00E94781F0EC006311C4509F097
:1011E0008FC08091D605882309F478C365E389E12F
:1011F00096E00E946B1F0E94EC195EC00F3D2CE52B
:10120000120709F44AC040F401155CE5150799F08E
:1012100001301C4579F174C00C359DE5190709F4BE
:1012200047C00D35ADE51A07D9F10B351D4509F05D
:1012300067C081E03EC00E9484150E940C230E947A
:10124000361F8C0163E070E085E692E00E9468271B
:10125000C8010E94271F8A3F910538F4EFE9FFE09B
:101260003197F1F700C00000F3CF0E94E5220E9401
:10127000DD1E22C08091AF06982F9095917090FB53
:1012800080F98093AF06992319F089EE91E002C0AE
:1012900087ED91E00E9487030FC00E9474190CC073
:1012A0008091790682FB882780F991E0892701C027
:1012B00080E00E94831A24C080915906877009F447
:1012C0000FC3D70112968C91882309F409C380912A
:1012D000790682FD05C382E0AD960FB6F894DEBFB5
:1012E0000FBECDBFDF91CF911F910F91FF90EF9077
:1012F000DF90CF90BF90AF909F908F900C94661A24
:10130000D70112968C9112970C911196DC9088233C
:1013100059F0802F9D2D0E949D12182F682F802F2D
:101320009D2D0E94FF1405C0802F9D2D0E94D31477
:10133000182FBCE31B9FF00111241CE0D19EE00D8F
:10134000F11D1124E00FF11DEE0FFF1FEF5CFC4FAC
:10135000859194910E94DA178C01982ED7011296EC
:10136000DC9012971596AC90A2943FE0A322809156
:1013700059068770B9F0DD20A9F0812F807F803475
:1013800021F080E2800F883068F08091790682FD3C
:1013900009C082E00E94661A809159068770CC24A9
:1013A000C3948111C12CB12EB2949FE0B9228B2D30
:1013B00090E08C30910508F054C2FC01EA5AFF4FCE
:1013C0000C944A2E812F807F1F70882311F0129574
:1013D000107FDD20B9F0112309F430C280E2800FC4
:1013E000883010F0911006C080916306182B10937E
:1013F000630605C080916206182B109362060E9456
:10140000EC191CC2802F0E94A015112309F429C2D7
:10141000005E083078F1992069F11095809162069C
:1014200018231093620629C0812F807F1F7080329D
:1014300011F01295107F992021F0B1E09B16D9F19F
:1014400049C08091790682FF1BC0DD2069F011231D
:1014500039F080916306182B109363060E94EC19F3
:1014600080E00E94F715FDC180E00E94A0151123C5
:1014700009F4F7C1812F0E94E5190E94EC19F1C10E
:10148000DD2081F080916406AA2051F0E1E0AE12E7
:1014900007C0182B181709F4E4C110936406E1C1C2
:1014A000812B10C0AA2021F0F1E0AF1609F4D9C1B8
:1014B0000E94DF192AC0DD2041F005E00A1508F47A
:1014C000D0C1812F0E949615CCC124E02A1508F4C2
:1014D000C8C11BC0DD2061F0AA2099F3D701159681
:1014E0008C91159780FFAAC18F7015968C93E9CFC8
:1014F000AA2059F0093309F0B1C1BFEFE7EEF3E0DC
:10150000B150E040F040E1F7A7C1812F0E948F1554
:10151000A8C1812F86958695837019F0813059F086
:10152000A0C1DD2019F0C801937002C080E090E0F6
:101530000E94A81F9CC1DD2019F0C801937002C051
:1015400080E090E00E94921F92C1812F837009F089
:1015500069C0D1108AC1902F929596959770990F76
:10156000990F802F8F70882E912CA12CB12C092ED1
:1015700004C0880C991CAA1CBB1C0A94D2F704FF57
:1015800012C04FE050E060E070E004C0440F551F0F
:10159000661F771F9A95D2F7DB01CA018095909557
:1015A000A095B09503C080E090E0DC0116951695FB
:1015B000412F4370423019F1C8F400916506109133
:1015C00066062091670630916806413059F08829F7
:1015D0009929AA29BB29BC01CD016023712382234B
:1015E00093230AC0802A912AA22AB32ABC01CD01E2
:1015F000682979298A299B290E947A1536C1882968
:101600009929AA29BB2900916506109166062091A7
:10161000670630916806BC01CD01602771278227DB
:101620009327EACFDD2019F0812F817001C08695C4
:10163000882309F41AC1902F929596959770990F67
:10164000990F802F8F70882E912CA12CB12C092EF0
:1016500004C0880C991CAA1CBB1C0A94D2F704FF76
:1016600012C04FE050E060E070E004C0440F551F2E
:10167000661F771F9A95D2F7DB01CA018095909576
:10168000A095B09503C080E090E0DC01169516951A
:10169000412F43704230D9F068F50091180710913E
:1016A000190720911A0730911B07413059F08829FA
:1016B0009929AA29BB29BC01CD016023712382236A
:1016C00093231EC0802A912AA22AB32A13C08829F4
:1016D0009929AA29BB29009118071091190720916F
:1016E0001A0730911B07BC01CD01602771278227A3
:1016F000932706C0BC01CD01682979298A299B2935
:101700000E942A15B2C01F70DD2039F0812F0E947F
:101710005915802F0E949615A8C0802F0E948F1502
:10172000812F0E943415A1C0802F22EF921609F458
:1017300043C0291538F030EF931659F051EF951644
:10174000B1F177C093EF9916F1F1A4EF9A1659F120
:1017500070C0DD2019F1B4E0BA1508F482C01F7121
:1017600081E090E0A0E0B0E0AC01BD0104C0440F16
:10177000551F661F771F1A95D2F780911807909111
:101780001907A0911A07B0911B078A019B0108272E
:1017900019272A273B27C901B80129C025E02A15A6
:1017A00008F45FC0DCCF8091790682FF23C0DD2082
:1017B00029F0812F8F7130C0DD20D9F3812F8F71F7
:1017C0000E9434154EC0DD2079F01F7181E090E059
:1017D000A0E0B0E0BC01CD0104C0660F771F881FF8
:1017E000991F1A95D2F703C060E070E0CB010E9408
:1017F0002A1537C0DD2099F01F71812F0E945915DD
:101800008091790682FD07C038E0139FC001112442
:10181000836080935906812F0E94591522C081E070
:101820000E94661A51E05A15E0F482E00E94661A9E
:1018300018C0DD2029F0AA2009F4BBCF802F11CEDB
:10184000AA2009F4BBCF893349F48FEF97EEA3E0C8
:1018500081509040A040E1F700C00000802F0E941E
:10186000A01588EF8B0D843010F40E94BE1FCC2091
:10187000A9F08091590680FD11C0F701128285956B
:10188000859585950E945915C7010E94290480916C
:1018900059068595859585950E94341585E0F70153
:1018A000DE01949601900D928A95E1F78CA19DA19D
:1018B0000E94D3149DA10CE3809FF00111241CE031
:1018C000919FE00DF11D11248CA1E80FF11DEE0F89
:1018D000FF1FEF5CFC4F8591949102C069E287CCB9
:1018E000AD960FB6F894DEBF0FBECDBFDF91CF919E
:1018F0001F910F91FF90EF90DF90CF90BF90AF902E
:101900009F908F9008958091E90587FF11C0809185
:10191000E80082FD05C08091E7058111F8CF11C074
:101920008091E8008B770BC08091E705882349F010
:101930008091E80080FFF8CF8091E8008E77809357
:10194000E8000895982F973068F59093E90098176C
:1019500039F07091EC002091ED005091F00003C03F
:10196000242F762F50E021FD02C09F5FECCF3091F5
:10197000EB003E7F3093EB003091ED003D7F3093E4
:10198000ED003091EB0031603093EB007093EC0090
:101990002093ED005093F0002091EE0027FDE5CF5D
:1019A00080E008958F708093E90081E00895209190
:1019B000EF053091F0052617370748F061157105DE
:1019C00039F42091E8002E772093E80001C0B90196
:1019D000FC0120E06115710579F18091E70588230C
:1019E000F1F18530F1F18091E80083FD3CC08091F8
:1019F000E80082FD2EC08091E80080FFEBCF2091AF
:101A0000F3008091F20090E0922B6115710551F086
:101A10008830910538F421912093F10061507109CB
:101A20000196F3CF21E0089709F020E08091E800CB
:101A30008E778093E800CECF2111CFCF0AC080915E
:101A4000E705882361F0853061F08091E80083FD2F
:101A50000AC08091E80082FFF2CF80E0089582E022
:101A6000089583E0089581E0089508959FB7F8945C
:101A70001092D8059FBF9091E705943009F057C0A8
:101A80009091E9009F703091EC00232F217030FD80
:101A900020E8922B23E02093E9002091EB0020FF27
:101AA00043C02091EE0027FF3FC02091D70522239D
:101AB00021F02091E80025FF37C01092D70526E0DD
:101AC0003091E80035FD15C03091E705343061F5FF
:101AD0003091EB0035FD28C0215021F481E0809346
:101AE000D70522C0EFE9FFE03197F1F700C0000011
:101AF000E7CF8093F1008091E80085FD0AC08091D6
:101B0000E80080FFFCCF8091E8008E778093E800AA
:101B100006C08FB7F89421E02093D8058FBF9F703F
:101B20009093E90080E008959F709093E9008FEF13
:101B30000895BC0184E00C94B21EBC0183E00C94B7
:101B4000B21E1F93CF93DF93CDB7DEB7AA970FB620
:101B5000F894DEBF0FBECDBFE9EEF5E08091F10055
:101B6000819345E0E13FF407C9F78091EA058330AE
:101B700009F461C030F4813071F0823009F49BC007
:101B8000B2C08A3009F487C08B3009F46CC0893048
:101B900009F0A9C020C08091E905813A09F0A3C0ED
:101BA0008091E800877F8093E8008091ED05909117
:101BB000EE05892B21F468E08DED95E003C060E02F
:101BC00080E090E070E00E94D70C8091E8008B7775
:101BD0008093E80088C08091E905813209F083C0D4
:101BE0008091ED059091EE05029708F07CC0809100
:101BF000E800877F8093E8008091E80082FD05C0BF
:101C00008091E7058111F8CF6EC02091F30080919B
:101C1000F20090E0922B029731F48091F100813034
:101C200011F0863021F48091F1008093DC058091E1
:101C3000E8008B7754C08091E905813A09F053C0E0
:101C40008091ED059091EE05892B09F04CC08091B3
:101C5000E800877F8093E8008091E80080FFFCCF58
:101C600080917D0237C08091E9058132E1F5809154
:101C7000ED059091EE05892BB1F58091E800877F05
:101C80008093E8000E94830C8091EB0580937D0295
:101C90000E94841528C08091E905813221F5809148
:101CA000E800877F8093E8000E94830C8091EC0518
:101CB0008093DB0518C08091E905813AA1F48091F9
:101CC000E800877F8093E8008091E80080FFFCCFE8
:101CD0008091DB058093F1008091E8008E778093FE
:101CE000E8000E94830C8091E80083FFDAC18091B4
:101CF000E9059091EA05492F50E04A30510508F076
:101D0000D0C1FA01EE59FF4F0C944A2E803821F0D1
:101D1000823809F0C6C108C08091E5059091E605BA
:101D2000992389F082600FC08091ED058F70873014
:101D300008F0B7C18093E9008091EB0085FB88270C
:101D400080F91092E9009091E800977F9093E80065
:101D50008093F1001092F10070C1282F2D7F09F0BF
:101D6000A0C1882319F0823061F09BC18091EB05FE
:101D7000813009F096C1933009F080E08093E60548
:101D80002EC08091EB0581112AC08091ED058F70E6
:101D90002FEF280F263008F084C18093E9002091AE
:101DA000EB0020FF1CC0933021F48091EB00806297
:101DB00014C09091EB0090619093EB0021E030E033
:101DC000A90102C0440F551F8A95E2F74093EA002B
:101DD0001092EA008091EB0088608093EB001092F3
:101DE000E9008091E800877F8093E8000E94830CDF
:101DF00058C1811156C11091EB051F778091E30006
:101E00008078812B8093E3008091E800877F809326
:101E1000E8000E94830C8091E80080FFFCCF809155
:101E2000E30080688093E300111102C082E001C0EA
:101E300083E08093E70535C18058823008F031C1D6
:101E40002091EB053091EC052C3D53E0350779F5F9
:101E500083E08A838AE289834FB7F894DE01139680
:101E600020E03EE051E2E32FF0E050935700E49190
:101E700020FF03C0E295EF703F5FEF708E2F90E080
:101E8000EA3010F0C79601C0C0968D939D932F5FE6
:101E9000243149F74FBF8091E800877F8093E800A5
:101EA0006AE270E0CE0101960E94D70CB5C0809125
:101EB000ED059091EE05432F552743305105A9F0CC
:101EC00068F44130510509F4FBC04230510509F076
:101ED000E8C08BE590E0E2EAF2E04BC04132510508
:101EE00029F14232510589F1DCC0C90199278130BD
:101EF0009105A1F058F0029709F0D3C0EFE0F3E0AC
:101F0000E4918E2F90E0EFE0F3E030C0EDE2F3E0FB
:101F1000E4918E2F90E0EDE2F3E028C0E1E2F3E0FF
:101F2000E4918E2F90E0E1E2F3E020C08330910550
:101F300008F0B7C0880F991FFC01E65CFA4F0190CA
:101F4000F081E02D89E090E014C08330910508F025
:101F5000A8C0FC01EE0FFF1FEC5CFA4F0190F0816E
:101F6000E02DDC01AF5CBA4F8C9190E0009709F452
:101F700098C02091E800277F2093E8002091EF058A
:101F80003091F0058217930708F49C0140E0211579
:101F9000310589F18091E705882309F43DC085303A
:101FA000D9F18091E80083FD37C08091E80082FD7F
:101FB0002FC08091E80080FFEACF4091F30080912C
:101FC000F20090E0942B2115310559F088309105ED
:101FD00040F444914093F10031962150310901962B
:101FE000F2CF41E0089709F040E08091E8008E7759
:101FF0008093E800CCCF4111CDCF0AC08091E70596
:10200000882351F0853041F08091E80083FD04C0C1
:102010008091E80082FFF2CF8091E8008B77809377
:10202000E8003FC08038E9F58091E800877F809321
:10203000E8008091E8058093F1008091E8008E77B8
:10204000D3CE81112EC08091EB059091EC0599279C
:1020500002973CF58091E800877F8093E80010911B
:10206000EB051093E8050E94830C111106C08091C6
:10207000E30087FD02C081E001C084E08093E705B2
:1020800042E061EC81E00E94A20C42E261EC82E05D
:102090000E94A20C42E261EC83E00E94A20C8091BB
:1020A000E7058091E80083FF10C08091E800877FFA
:1020B0008093E8008091EB0080628093EB0005C084
:1020C00082E190E0EDEFF2E054CFAA960FB6F894DB
:1020D000DEBF0FBECDBFDF91CF911F9108951F923C
:1020E0000F920FB60F9211242F933F934F935F934C
:1020F0006F937F938F939F93AF93BF93CF93DF9310
:10210000EF93FF93C091E900CF708091EC00D82F3E
:10211000D17080FDD0E81092E9008091F000877FB7
:102120008093F00078940E94A10D1092E9008091B4
:10213000F00088608093F000CD2BCF70C093E90051
:10214000FF91EF91DF91CF91BF91AF919F918F91CF
:102150007F916F915F914F913F912F910F900FBEA3
:102160000F901F901895E8EDF0E080818E7F8083BE
:102170001092E2001092DA001092E100A0EEB0E0BE
:102180008C9181608C9380818F77808319BCA7EDBF
:10219000B0E08C918E7F8C9380818F7E80831092B3
:1021A000DA050895CF92DF92EF92FF920F931F937B
:1021B000CF93DF93C8EDD0E088818F7E8883E7EDF1
:1021C000F0E080818160808384E082BF81E0809341
:1021D000DA0588818E7F888302EE10E0F801108294
:1021E0001092DA0081EEC82ED12CF601108288817F
:1021F0008F77888388818068888388818F7D8883B2
:1022000019BC1092E7051092E8051092E6051092AD
:10221000E50590EEE92EF12CF70180818B7F80831C
:1022200088818160888342E060E080E00E94A20CA7
:10223000F60180818E7F8083F801808181608083B8
:10224000808188608083F70180818E7F8083888190
:1022500080618883DF91CF911F910F91FF90EF9064
:10226000DF90CF9008951F920F920FB60F92112416
:102270002F933F934F935F936F937F938F939F938E
:10228000AF93BF93EF93FF938091E10082FF49C02A
:102290008091E20082FF45C08091E1008B7F8093B6
:1022A000E1002091D9052F5F822F62E30E94162E54
:1022B000992319F02093D90534C01092D905809143
:1022C000D805882371F18091E705843041F580912C
:1022D000E9008F702091EC00922F917020FD90E822
:1022E000892B93E09093E9009091EB0090FF14C04C
:1022F0009091EE0097FF10C09091E80095FF03C009
:102300001092F100F9CF9091E80090FF05C09091F4
:10231000E8009E779093E8008F708093E900109218
:10232000D8058091DA0080FF32C08091D80080FF0C
:102330002EC08091DA008E7F8093DA008091D900E0
:1023400080FF1CC080E189BD82E189BD09B400FE27
:10235000FDCF81E08093E7058EE892E00E9487033D
:102360008091DA05811113C00E94B3100E94D2102F
:102370008091E20084608093E20009C019BC109251
:10238000E70582E992E00E9487031092DA058091C6
:10239000E10080FF1BC08091E20080FF17C08091A8
:1023A000E2008E7F8093E2008091E2008061809362
:1023B000E2008091D80080628093D80019BC85E04B
:1023C0008093E70586E992E00E9487038091E1000F
:1023D00084FF34C08091E20084FF30C080E189BD79
:1023E00082E189BD09B400FEFDCF8091D8008F7DC8
:1023F0008093D8008091E1008F7E8093E1008091EE
:10240000E2008F7E8093E2008091E2008160809301
:10241000E2008091E805882311F084E007C08091F4
:10242000E30087FD02C081E001C083E08093E705FF
:102430008AE992E00E9487038091E7058091E1009C
:1024400083FF2BC08091E20083FF27C08091E100D1
:10245000877F8093E10082E08093E7051092E80592
:102460008091E1008E7F8093E1008091E2008E7F79
:102470008093E2008091E20080618093E20042E07C
:1024800060E080E00E94A20C8091F0008860809360
:10249000F0008EE992E00E948703FF91EF91BF91D7
:1024A000AF919F918F917F916F915F914F913F91EC
:1024B0002F910F900FBE0F901F9018952091E40060
:1024C0003091E50095E64091EC00842F817040FF4B
:1024D00023C08091E80080FD1DC08091E70588231E
:1024E00099F0853099F08091EB0085FD11C0409105
:1024F000E4005091E5002417350729F3915011F0BD
:102500009A01E1CF84E0089582E0089583E0089580
:1025100081E0089580E008954091E80042FFDDCF1A
:10252000089580E090E00E94A81F80E090E00E9463
:10253000921F109262060C94EC198F929F92AF92A8
:10254000BF92DF92EF92FF920F931F93CF93DF938F
:102550008090180790901907A0901A07B0901B0759
:102560004091650650916606609167067091680615
:10257000842A952AA62AB72ACFE1D0E02CE0929FA0
:10258000700111249CE3D92E082F10E0D501C4015D
:102590000C2E04C0B695A795979587950A94D2F707
:1025A00080FD04C0219790F780E014C0DC9EF0010C
:1025B000DD9EF00D1124EE0DFF1DE00FF11FEE0F5B
:1025C000FF1FEF5CFC4F859194910E94DA170197F1
:1025D00049F38C2FDF91CF911F910F91FF90EF90D6
:1025E000DF90BF90AF909F908F900895CF93DF932F
:1025F000EC010E949D122CE3829FC0011124FC017A
:102600002CE0D29FE00DF11D1124EC0FF11DEE0F17
:10261000FF1FEF5CFC4F859194910E94DA17DF91C8
:10262000CF910895FC01808191810E94F6129295CC
:102630009F70963079F010F4925001C09A50923009
:1026400068F4803F69F018F4883E40F409C0843F84
:1026500029F406C0883E20F0813F11F080E0089503
:1026600081E008959F92AF92BF92CF92DF92EF9256
:10267000FF920F931F93CF93DF93CDB7DEB7619790
:102680000FB6F894DEBF0FBECDBF8C0185E0F80118
:10269000DE011D9601900D928A95E1F7F801E28026
:1026A00090912106609122064091240650912506C2
:1026B0004115510531F06F3F31F481E09F3F19F42E
:1026C00003C081E001C080E0F82FF1709F2E80FDF3
:1026D0001AC1F80130812181C380D48081E2A82E03
:1026E00086E0B82EF0902306F601E41BF50BFF20E0
:1026F00009F4C6C080912606E83CF10508F091C0B7
:10270000482F407F09F050C0621311C093130FC0CF
:10271000FE2CE1100CC08F70806180932606C501ED
:102720000E94290480912606F801858329C1CD28BD
:1027300031F02F3F31F481E03F3F19F403C081E0D5
:1027400001C080E080FD03C081E08E2502C080E0F2
:1027500090E0F82FF170FF2E80FF1CC0809158068A
:102760004091270656E0841709F4E8C090E0589F8E
:10277000F001599FF00D1124E85DF94F6181261396
:1027800006C06081631303C06281E61203C0019634
:102790008770E9CFFE2CEE2009F4F2C08091260666
:1027A00081608093260649C0621306C0931304C05B
:1027B000E11002C0F80186C0C8010E9412138823EC
:1027C00051F1EE2041F120912606822F82958F70E3
:1027D00090E0029774F080912106909122069887EC
:1027E0008F831986DB86CA862C87CE0107960E94C6
:1027F000290486E0F801A1E2B6E001900D928A95E5
:10280000E1F70E94BC1A0AC06217C9F0C8010E9411
:10281000121381111EC0C8010E942904FF24F394E1
:10282000AFC0482F407F81F781E296E00E942904E3
:1028300086E0F50111928A95E9F7F12CA1C0931376
:10284000E5CFE110E3CFF8018583C8010E94290498
:1028500054C0EE2001F320912606822F82958F70BE
:1028600090E0029734F280912106909122069A839B
:1028700089831B82DD82CC822E83CE010196B7CF65
:10288000E83CF105D0F5FE2CEE2029F2621327C0BA
:10289000931325C02091260620FD18C0822F829513
:1028A0008F70482F50E04115510581F0F8012583C4
:1028B0004F30510541F08F5F982F9295907F822F76
:1028C0008F70892B8583C8010E94290486E0F80156
:1028D000A1E2B6E001900D928A95E1F751C0C801DE
:1028E0000E941213811185CF80912606816080930A
:1028F0002606C8010E94290443C086E0F501119212
:102900008A95E9F73DC0EE2009F485CFC8010E9401
:102910001213F82E882309F47ECF86E0F801A1E295
:10292000B6E001900D928A95E1F780912106909191
:1029300022060E94F6120E94BC1A22C03D872E87F2
:102940008D859E850E94F612292F22952F702230A8
:1029500028F49F7039F0811105C00BC0243028F491
:102960009F7049F4805E883020F0C8010E942904DD
:102970009F2CF92C05C0F8019581907F99F7F9CF2C
:102980008F2D61960FB6F894DEBF0FBECDBFDF91DD
:10299000CF911F910F91FF90EF90DF90CF90BF905C
:1029A000AF909F9008952CE0929F800D1124682F86
:1029B000669566956695982F977085E0689FB0013B
:1029C000112440E050E080E0FB01E40FF51FEF50E0
:1029D000FA4F208130E0092E02C0369527950A94DF
:1029E000E2F721703327042E01C0220F0A94EAF780
:1029F000822B4F5F5F4F4530510531F708952CE032
:102A0000929F800D1124E82FE695E695E695877054
:102A100051E001C0550F8A95EAF785E0E89FF00183
:102A20001124EF50FA4F20E030E070E04081CB01FC
:102A3000022E02C0969587950A94E2F781708195DF
:102A400084278523842781932F5F3F4F25303105CD
:102A500069F70895609318077093190780931A0710
:102A600090931B070C9491120F931F9341E050E039
:102A700060E070E004C0440F551F661F771F8A9501
:102A8000D2F7409550956095709580911807909178
:102A90001907A0911A07B0911B078A019B0108230F
:102AA00019232A233B23C901B8011F910F910C94CC
:102AB0002A150F931F9341E050E060E070E004C0DE
:102AC000440F551F661F771F8A95D2F7809118070C
:102AD00090911907A0911A07B0911B078A019B01D9
:102AE000082B192B2A2B3B2BC901B8011F910F91E1
:102AF0000C942A15609365067093660680936706AA
:102B0000909368060C9491121092630686E0EBE1B4
:102B1000F6E0DF011D928A95E9F70C949112882363
:102B200021F00E94E5190C94EC190895882339F0DE
:102B300090916306892B809363060C94EC19089599
:102B4000882309F453C0682F823869F40E94BE1F9D
:102B500081FF4CC069E389E196E00E94781F0E94E2
:102B6000EC1969E30EC0833891F40E94BE1F80FF08
:102B70003DC063E589E196E00E94781F0E94EC1950
:102B800063E589E196E00E946B1F0C94EC19843890
:102B900069F40E94BE1F82FF29C067E489E196E0C4
:102BA0000E94781F0E94EC1967E4EBCF8CEF860F30
:102BB000813A38F380E2860F883048F4677081E00C
:102BC00001C0880F6A95EAF70E94E519DECF8BE510
:102BD000860F833020F480E090E00C94A81F685AA0
:102BE000673120F480E090E00C94921F0895CF9319
:102BF000882309F496C0C82F8238B1F40E94BE1F02
:102C000081FD8FC069E389E196E00E94781F0E94F0
:102C1000EC192FEF81EE94E0215080409040E1F7D5
:102C200000C0000069E317C08338E1F40E94BE1FB2
:102C300080FD77C063E589E196E00E94781F0E94DD
:102C4000EC192FEF81EE94E0215080409040E1F7A5
:102C500000C0000063E589E196E00E946B1FCF9100
:102C60000C94EC198438B1F40E94BE1F82FD59C047
:102C700067E489E196E00E94781F0E94EC192FEF2B
:102C800081EE94E0215080409040E1F700C00000C8
:102C900067E4E1CF8CEF8C0F813A80F4EBE1F6E052
:102CA00081E296E02191C217A1F18E179F07D1F71B
:102CB0006C2F89E196E00E94781FD1CF80E28C0FC3
:102CC000883068F4C77081E090E001C0880FCA9531
:102CD000EAF790916306892B80936306C0CFEBE5FA
:102CE000EC0FE33040F4F0E0E05CFA4F808190E0DC
:102CF000CF910C94A81FC85AC73198F4EC2FF0E07C
:102D0000EE0FFF1FED5BFA4F80819181CF910C9404
:102D1000921F6C2F89E196E00E946B1F0E94EC19B4
:102D2000C7CFCF9108959091780692FF0DC0282FBC
:102D30002871283019F4877F846006C0282F2471F9
:102D4000243011F48B7F886093FF0DC0282F2871E9
:102D5000283119F4877E846106C0282F247124311C
:102D600011F48B7E88612091790620FF0DC0382FE9
:102D70003871383019F4877F816006C0382F31717F
:102D8000313011F48E7F886021FF0DC0282F28710B
:102D9000283119F4877E816106C0282F21712131E5
:102DA00011F48E7E886194FD877E0895F894E82F53
:102DB000E295EF70F0E031A1282F2F7081E090E0D4
:102DC00001C0880F2A95EAF7982F9095932391A335
:102DD00092A1892B82A3789408958F929F92AF92AB
:102DE000BF92CF92DF92EF92FF920F931F93CF93F8
:102DF000DF93CDB7DEB72A970FB6F894DEBF0FBECC
:102E0000CDBFAE014F5F5F4F7A018AE0FA011192A8
:102E10008A95E9F701E715E06A01AA24A394B12C89
:102E2000F80180818F3F09F447C0F894E82FE295BC
:102E3000EF70F0E021A18F70A50102C0440F551F73
:102E40008A95E2F7CA01922F982B91A392A18095BF
:102E5000892382A3789400C0E6E7F5E021E030E022
:102E6000812C912C41914F3F89F0A42FA295AF70F6
:102E7000B0E090968C9190E04F7002C09595879548
:102E80004A95E2F780FD02C0C90102C080E090E0EF
:102E9000882A992A220F331F55E0E238F50711F7E7
:102EA000F80180818F3F11F00E94D616F0EAFA9562
:102EB000F1F7F601918280820F5F1F4FF2E0CF0E93
:102EC000D11C45E00637140709F0AACF4AE050E0CC
:102ED000B7018EE696E00E94502E11E0009709F4AB
:102EE00010E0892B89F08AE0F701AEE6B6E00190A8
:102EF0000D928A95E1F781E080936B060E94361F60
:102F000090936A068093690680916B06882391F1FD
:102F10008091690690916A060E94271F059750F1DB
:102F200080916E0690916F0690937B0680937A064F
:102F3000809170069091710690937D0680937C0637
:102F4000809172069091730690937F0680937E061F
:102F50008091740690917506909381068093800607
:102F600080917606909177069093830680938206EF
:102F700010926B0680916C0690916D06892B31F052
:102F80000E94E52210926D0610926C06812F2A96FF
:102F90000FB6F894DEBF0FBECDBFDF91CF911F916A
:102FA0000F91FF90EF90DF90CF90BF90AF909F90E8
:102FB0008F900895CF93DF938238910569F1B0F433
:102FC0008133910509F46FC048F48932910509F401
:102FD00065C08A32910509F46BC08AC085339105BA
:102FE00009F457C089339105B9F082C0833E910539
:102FF00071F138F4803E9105B1F0823E910511F1F6
:1030000077C0863E9105B9F1873E9105C9F1843EAE
:10301000910509F06DC024C02091780620FD53C0B1
:1030200021FD51C065C08091780680FD46C0809129
:10303000790680FF48C08091780684FD3FC183EE09
:1030400090E03EC18091780682FF3AC0F4CF809133
:10305000780682FD35C08091790680FD34C0EBCFC3
:103060008091790681FF35C08091780684FD26C164
:1030700087EE90E025C18091780683FF27C0F4CFCA
:103080008091780683FD22C08091790681FD21C060
:10309000EBCF8091780685FD1FC021C08091780616
:1030A00085FD1DC019C08091780686FD1BC01DC01E
:1030B0008091780686FD19C015C089E390E000C1B3
:1030C00082EE90E0FDC080EE90E0FAC086EE90E0E7
:1030D000F7C084EE90E0F4C089E290E0F1C085E3AF
:1030E00090E0EEC08AE290E0EBC081E390E0E8C0BF
:1030F000811532E5930708F069C0811541E5940711
:1031000028F0982F8827816F906ADAC0883E910551
:1031100068F5803E910508F0D3C0883A9105B8F46F
:10312000853A910548F0855AE82FF0E0E05CFA4FC7
:10313000808190E09064C4C08130910509F4BBC0E7
:1031400008F4BCC08430910508F4B8C0B9C08F3B06
:10315000910508F0B3C0885AE82FF0E0EE0FFF1F8A
:10316000ED5BFA4F808191819464AAC0811520E5BE
:103170009207F0F09C0174E0369527957A95E1F777
:10318000922F9370482F437021E030E002C0220F4D
:10319000331F4A95E2F73C68392B8F70982F96952C
:1031A000969540E2949FC0011124822B932B88C0F6
:1031B000811530E4930718F09F70906A81C09C01DC
:1031C0003A9521153F4108F47BC078C0EC01C11548
:1031D00086E5D807E8F5C11525E5D20748F08C2F1C
:1031E0000E9493168F7190E0982F8827906268C094
:1031F000C11534E5D30728F09C2F8827846F906A87
:103200005FC0AE01437055272C2F26952695C1151A
:10321000D34578F481E090E002C0880F991F4A9569
:10322000E2F740E2249F90011124822B932B9C68AB
:1032300047C081E090E002C0880F991F4A95E2F7ED
:1032400040E2249F90011124822B932B9A6838C06E
:10325000C1152AE5D207F8F4C11539E5D30790F076
:103260008C2F8F700E94931694E0D695C7959A95EF
:10327000E1F7CF70D0E0DC2FCC27D0699E01282B5E
:10328000C9011EC0C11548E5D407C0F09C2F88278E
:10329000806F906A15C0CE0190568115904270F4EF
:1032A0008D2F8F710E949316282F2F71CE01992791
:1032B0009062922B05C081E090E002C080E090E037
:1032C000DF91CF910895CF9384E090E00E944F2941
:1032D000C82F82E290E00E944F292C2F30E0A901F4
:1032E000582BCA01CF91089569EE7EEF80E090E0FF
:1032F0000E947B2960E082E090E00E945D2960E00E
:1033000083E090E00E945D291092650610926606A7
:10331000109267061092680660E084E090E00E94D8
:103320005D2960E082E290E00E945D2960E085E036
:1033300090E00E945D2960E086E090E00E945D29B7
:103340006FEF87E090E00E945D2940E050E0BA0115
:1033500088E090E00E946F2960E08DE090E00E949C
:103360005D2940E050E0BA0188E190E00E946F29B9
:1033700060E087E190E00E945D2940E050E0BA0102
:103380008CE190E00E946F2960E070E080E290E0C4
:103390000E947B2940E050E0BA0188E190E00E9461
:1033A0006F2940E050E0BA018FE090E00E946F2961
:1033B00040E050E0BA0183E190E00C946F298091E5
:1033C00064068111109264060895809590916306B9
:1033D0008923809363060895EF92FF920F931F93C2
:1033E000CF939091630680916206982B9093190673
:1033F00080916406882389F0892B80931906EBE17C
:10340000F6E097E080E0915029F021912223D9F352
:103410008F5FF9CF81110E94DF1948E050E06AE523
:1034200076E089E196E00E94502E892B09F448C08D
:1034300088E0E9E1F6E0AAE5B6E001900D928A9510
:10344000E1F7E091B606F091B7063097C9F1028036
:10345000F381E02D89E196E009958091AF0682FF26
:103460002FC080FF04C08EE196E00E94870309E12F
:1034700016E0C8E088E1E82E86E0F82E8091AF06DD
:1034800080FF0CC0F80180811F928F93FF92EF9212
:103490000E9420040F900F900F900F90C1500F5F6B
:1034A0001F4FC111EBCF8091AF0680FF09C086E1AD
:1034B00096E0CF911F910F91FF90EF900C948703AE
:1034C000CF911F910F91FF90EF9008952091590691
:1034D0008095822380935906982F977099F430E055
:1034E000482F082E000C550B2417350759F09091E2
:1034F000790692FD07C08595859585950E943415BE
:10350000109259060895CF93DF93C0917906C2FBBC
:10351000992790F9981719F1D82F80FBC2F9C09319
:1035200079066091780684E090E00E945D296C2F16
:1035300082E290E00E945D2982E00E94661A8091FA
:10354000AF0680FF0CC01F92DF9381E096E09F934F
:103550008F930E9420040F900F900F900F90DF9197
:10356000CF9108958091580690912706891719F0F8
:103570008F5F8770FBCF08950F931F93CF93DF93D7
:103580008091260682958F7009F05DC08091230698
:10359000882309F458C0809158061091270660913D
:1035A000210670912206C0912406D091250691E053
:1035B0006F3F09F090E0292F06E0811709F443C01E
:1035C000209721F07F3F21F030E003C031E001C0BF
:1035D000322F90E030FD34C0089FF001099FF00DBC
:1035E0001124DF01A85DB94F11963C911197371353
:1035F00027C03C91361324C012963C91129731118A
:103600001FC013964D915C9114974C1B5D0B483C69
:103610005105B0F4809126068F7080618093260654
:10362000E35DF94F80818F708061808381E296E055
:103630000E942904DF91CF911F910F910C94B21A2F
:1036400001968770BACFDF91CF911F910F910895A6
:1036500062E070E08CEB92E00E9468272FEF81EE31
:1036600094E0215080409040E1F700C000000E94AB
:10367000E5226091D1066E7F6093D10687E090E0ED
:103680000C945D296091D10661606093D10687E05A
:1036900090E00E945D2962E070E08CEA92E00C9478
:1036A00068278091D006811144C080E090E00E949C
:1036B0005729893E9E4F11F00E94741987E090E0CF
:1036C0000E944F298093D106E7EDF6E080E090E07C
:1036D000A0E8BFEB1182108282839383A483B58319
:1036E00017821682389627E0E731F20799F7809122
:1036F000D00681110CC00E948B213E9A82E08093FB
:1037000090008AE18093910081E08093D0060E942E
:10371000E5228091D10680FF06C064E070E08CE86D
:1037200092E00E9468270E94361F9093C5068093FE
:10373000C4060895682F70E065547109072E000CC7
:10374000880B990B0E94102B20E030E040E451E4FC
:103750000E94662A9B01AC0160E070E080E090E48A
:103760000E948F2C20E030E04CED53E40E94222C8C
:1037700008950E949A1B4FEF5FEF0C949621CF9310
:10378000DF93CDB7DEB72B970FB6F894DEBF0FBE31
:10379000CDBF84B7877F84BF0FB6F894A89580917A
:1037A0006000886180936000109260000FBE90E01E
:1037B00080E80FB6F89480936100909361000FBE8B
:1037C00085B7806885BF85B7806885BF86E39DE043
:1037D0009093D3058093D2050E94B3100E94D2101B
:1037E0008091E20084608093E20078948091E70504
:1037F0008823A1F01091E9001F709091EC00892FAF
:10380000817090FD80E8182B1092E9008091E8000B
:1038100083FD0E94A10D1F701093E90082E084BD1A
:1038200093E095BD9AEF97BD80936E0001E715E098
:10383000B6E7EB2EB5E0FB2ED8018D918D018F3FC1
:1038400011F00E94D616E016F106B1F706E715E072
:10385000A2E8EA2EA5E0FA2EF80181918F018F3FB0
:1038600011F00E94D616E016F106B1F78AE0EAE7F9
:10387000F6E0DF01282F1D922A95E9F7EEE6F6E043
:10388000DF011D928A95E9F76E9A769A80E090E0C2
:103890000E945729893E9E4F11F00E94741982E0C0
:1038A00090E00E944F298093AF060E946319909385
:1038B0007906809378060E94ED16EFE3FCE93197D4
:1038C000F1F700C000000E94ED1680917A0680FF9B
:1038D00008C06FEF7FEF80E090E00E947B290E949C
:1038E000DD1E83E090E00E944F29682F70E080E0A9
:1038F00090E00E947A15279A2F988AE080938000A2
:1039000089E1809381008FEF9FEF909387008093F0
:1039100086000E944B210E94511B0E944B218EE782
:1039200092E09093B7068093B6068091E7058530C4
:1039300009F053C080E396E00E948703F0E4FF2E75
:1039400000E112E18091E705853009F040C08091E7
:10395000E705843041F180E00E9455200E94E52275
:103960001092BA0648E150E00FB6F894A89540933B
:1039700060000FBEF092600083B7817F846083BFD8
:1039800083B7816083BF7894889583B78E7F83BF28
:103990000FB6F894A89580916000886180936000CC
:1039A000109260000FBE8091E605882309F4CACF0B
:1039B0000E94ED16EAE7F6E081919191892B09F0DA
:1039C00037C184E896E08E179F07B1F7BBCF0E94FE
:1039D00084150E944B210E94BE1F0E94ED16882371
:1039E00059F08FB7F8944091BB065091BC06609196
:1039F000BD067091BE068FBF74E8472E76E0572E45
:103A0000EAE76E2EE6E07E2E00E010E00B87D301A1
:103A1000AD90BD903D01F201C190D1902F01CA241B
:103A2000DB24C114D104B1F40F5F1F4F0530110521
:103A300069F78FEF8E838F8318860E94361F81600F
:103A4000782F9A8789874E815F8168858A850E9451
:103A5000102878C08091AF0681FD05C080E0EE247B
:103A6000E394F12C49C084E496E00E9487035AE76E
:103A7000852E56E0952EE12CF12CFF92EF924FE32C
:103A800056E05F934F930E9420048CE396E00E94DF
:103A90008703D4018C9111962C90B2E08B0E911C6F
:103AA0000E94B828382E822D0E94B828232D30E09D
:103AB000322F2227F901E82BCF019F938F9346E302
:103AC00056E05F934F930E94200484E396E00E94A7
:103AD00087039FEFE91AF90A0FB6F894DEBF0FBE0D
:103AE000CDBFB5E0EB16F10441F6B8CF8F5FEE0C19
:103AF000FF1C8C3009F498CF97012C213D21232BFA
:103B0000A9F38983EB85EA83AE20BF2081E0AB284F
:103B100009F480E08B830E94361F8160782F9D839B
:103B20008C8349815A816B818D810E941028000FFE
:103B3000111FF801EC57F94F80819181E826F92691
:103B4000F182E0828091A206882309F444C080912A
:103B5000A0069091A106009781F40E94361F9093D1
:103B6000A1068093A00620919F0630E02115310523
:103B700071F480919E0690E00BC00E94271F209157
:103B80008A0230918B022817390738F324C0C90103
:103B90000197F901E257F94F10812091AD062223D8
:103BA00041F0FC01E257F94F80810E949A1B0E946C
:103BB0006A228091AD06882319F0812F0E94B91BDB
:103BC00080919F0690E0019660919E0670E00E94B1
:103BD000362E80939F060E94BE1F182F8091A30649
:103BE000181709F4A2CE1093A3068091AF0682FFA6
:103BF0009CCE80FF04C082E696E00E9487038091FD
:103C0000AF0680FF0CC01F921F938DE596E09F9337
:103C10008F930E9420040F900F900F900F9080912F
:103C2000AF0680FF82CE8BE596E00E9487037DCEB3
:103C300009BD19BD09B400FEFDCF8091D8008F7D6C
:103C40008093D8008091E00082608093E0008091B2
:103C5000E00081FDFCCF0E94841574CE0895809110
:103C6000DC050895CF92DF92EF92FF926B017C0109
:103C700020E030E0A9010E94612A811106C08091F4
:103C800090008F73809390003CC08091900080687A
:103C900080939000C092A506D092A606E092A70657
:103CA000F092A80620E030E040E051E4C701B60100
:103CB0000E94222C9B01AC0160E074E284E79BE44B
:103CC0000E94662A6B017C010E94DF2A7093970094
:103CD0006093960060918D0370E080E090E00E9418
:103CE000102BA70196010E94222C20E030E048EC26
:103CF00052E40E94662A0E94DF2A70939900609322
:103D00009800FF90EF90DF90CF900895CF93DF93CE
:103D100021E02093E9002FEF3091E800215035FD9C
:103D200006C035ED3A95F1F700002111F5CF20914D
:103D3000E80025FF14C0EC0140E050E068E070E0CE
:103D40000E94E4278091E8008E778093E80088E065
:103D5000FE01ADEDB5E001900D928A95E1F7DF919E
:103D6000CF9108958093BF067093C1066093C006FB
:103D70008091E705843001F582E08093E9008FEFC0
:103D80009091E800815095FD06C095ED9A95F1F768
:103D900000008111F5CF8091E80085FF0DC040E063
:103DA00050E063E070E08FEB96E00E94E4278091A2
:103DB000E8008E778093E800089581E08093E0002A
:103DC00080E28093D8001092C9008FE19EE40197B1
:103DD000F1F700C0000087E090EBDC0180931C0746
:103DE00090931D07A0931E07B0931F079CE088E1E6
:103DF0000FB6F894A895809360000FBE9093600072
:103E0000FFCF78941F920F920FB60F9211248F93C9
:103E10009F93AF93BF938091BB069091BC06A091F6
:103E2000BD06B091BE060196A11DB11D8093BB06D3
:103E30009093BC06A093BD06B093BE06BF91AF9110
:103E40009F918F910F900FBE0F901F9018959C011E
:103E50004FB7F8948091BB069091BC06A091BD0627
:103E6000B091BE064FBF821B930B08952FB7F894F5
:103E70008091BB069091BC06A091BD06B091BE0694
:103E80002FBF08951F920F920FB60F9211248F9398
:103E90009F93AF93BF938091BA06811113C0809115
:103EA000BB069091BC06A091BD06B091BE0641969E
:103EB000A11DB11D8093BB069093BC06A093BD06C7
:103EC000B093BE06BF91AF919F918F910F900FBE9F
:103ED0000F901F9018959C012A5F3F4FFC01428173
:103EE000461301C01282019682179307B9F708950D
:103EF0009C01FC0132969FEF80E04191461789F0CA
:103F00009F3F19F4411101C0982F8F5F8630A9F7A8
:103F10009F3F39F0F901E90FF11D97FDFA95628392
:103F2000089508952091B8063091B90628173907E9
:103F300071F09093B9068093B806E091B606F091BF
:103F4000B706309721F00084F185E02D099408959B
:103F50002091B4063091B5062817390771F0909377
:103F6000B5068093B406E091B606F091B706309797
:103F700021F00680F781E02D09940895E091B606BE
:103F8000F091B706309721F00190F081E02D09946F
:103F900080E00895EF92FF920F93CF93DF93C42FA9
:103FA000D22FFC0182818823D1F04093B3060E9476
:103FB000361F9093B2068093B10680E28C0F883052
:103FC00008F06DC0C77081E001C0880FCA95EAF79C
:103FD000DF91CF910F91FF90EF900C949615809107
:103FE000B30648134BC08091B1069091B2060E946F
:103FF000271F883C910508F041C0CD17C9F080E229
:104000008C0F883040F4C77081E001C0880FCA95DA
:10401000EAF70E948F1580E28D0F883048F481E026
:104020009D2F977001C0880F9A95EAF70E94961508
:10403000093319F0E12CF12C03C080E5E82EF12CB6
:10404000802F0E94F715E114F10451F08FE99FE0F1
:104050000197F1F700C0000091E0E91AF108F3CFF1
:10406000802F0E94A01580E28D0F8830C0F4D77099
:1040700081E001C0880FDA95EAF70AC080E28C0F70
:10408000883068F4C77081E001C0880FCA95EAF7EC
:10409000DF91CF910F91FF90EF900C948F15DF91EE
:1040A000CF910F91FF90EF9008958F929F92AF92D2
:1040B000BF92CF92DF92EF92FF920F931F93CF9315
:1040C000DF93843048F4811108C090918000977F7D
:1040D000909380002F9806C083E0909180009860B4
:1040E00090938000A0918600B0918700282F30E047
:1040F0000E94E52923E030E040E050E00E94C3291F
:104100000027122F232F342F012F122F232F332775
:1041100080918600909187006CE070E00E94222ED2
:104120006017710730F0C80169E070E00E94222E2C
:104130005EC08091860090918700E0908600F090AC
:104140008700E0918600F0918700C6E0D0E0BE01D4
:104150000E94222E060F171F211D311D48015901F3
:1041600085E0880C991CAA1CBB1C8A95D1F7C70155
:10417000BE010E94222E6F01E12CF12CA7019601B5
:10418000260F371F411D511DC501B4010E94C329CF
:1041900069017A01E0918600F0918700CA01B901B6
:1041A0000E94062E9B01AC01DF010E94B0299B01F9
:1041B000AC01C701B6010E94062EDC01CB012FE045
:1041C000B695A795979587952A95D1F70091860082
:1041D0001091870020E030E0081719072A073B07F5
:1041E00028F46091860070918700CB01BC01709328
:1041F0008D0060938C00DF91CF911F910F91FF9004
:10420000EF90DF90CF90BF90AF909F908F900895E8
:10421000682F86E090E00C945D299091B006892F7C
:104220008695869586958F5F8F719770843038F468
:10423000880F880F880F892B8093B00602C0909357
:10424000B0068091B006887F91E009F490E08091FB
:10425000B00690FB80F98093B0060E9408218091FF
:10426000AF0680FF11C08091B00686958695869531
:104270001F928F938DE696E09F938F930E94200468
:104280000F900F900F900F908091B00686958695B5
:1042900086950C94552080E090E00E945729893E35
:1042A0009E4F51F00E9474198091B006847089610C
:1042B0008093B0060E94082186E090E00E944F297A
:1042C0008093B006282F26952695269530E0243039
:1042D000310524F0877088618093B0068091B00624
:1042E00080FF04C086958695869501C080E00C9479
:1042F000552081E08093AE0668E070E08DE493E0A5
:104300000C94682781E08093AD0668E070E08DEC46
:1043100092E00C946827E1E7F0E080818D7F808354
:10432000E0E9F0E080818F73808308957F928F921F
:104330009F92AF92BF92CF92DF92EF92FF920F9334
:104340001F93CF93DF934B015C016A018091D106EB
:1043500080FFB2C08091D006811102C00E94511B23
:1043600020E030E0A901C501B4010E94612A87FF65
:1043700004C0B7FAB094B7F8B09470901707072D3F
:1043800010E0E801219743E0000F111F4A95E1F783
:10439000E12CF12CCF3FFFEFDF07D9F128E0E21A43
:1043A000F108F801EE0DFF1DE952F94F228133812A
:1043B00044815581C501B4010E94612A811127C041
:1043C0008E0133E0000F111F3A95E1F70952194FA2
:1043D0008091170790E00197C817D9070CF06CC0BF
:1043E000219688E0F8013896D80101900D928A95BF
:1043F000E1F70E94361FF8019187808782869386B5
:10440000A486B586D786C686085F1F4FE1CF219761
:10441000C1CF81E0870D893040F58093170781E097
:104420008093A4068093CF06C0911707D0E0219710
:104430000E94361FFE0123E0EE0FFF1F2A95E1F7D1
:10444000E952F94F9183808382829382A482B5825C
:10445000D782C6820E94361F9093D6068093D506D7
:104460008091CC02882341F113C088E08093170724
:1044700087ED96E028E0FC013896DC0101900D9272
:104480002A95E1F7089627E08F30920799F7C7CF72
:1044900080917100826080937100809190008068AB
:1044A000809390008091CF06882321F00E94F7240A
:1044B0000E94321E1092CC02DF91CF911F910F917A
:1044C000FF90EF90DF90CF90BF90AF909F908F9034
:1044D0007F900895CF92DF92EF92FF920F931F93F8
:1044E000CF93DF936B017C0120E030E0A9010E94B3
:1044F000612A87FF04C0F7FAF094F7F8F0948091EE
:10450000CF06882309F458C08091D006811102C0DB
:104510000E94511B07ED16E0C7E0D0E0F80122AD84
:1045200033AD44AD55ADC701B6010E94612A81117A
:104530002BC083E0CC0FDD1F8A95E1F7C952D94F1C
:104540001982188280E090E0A0E8BFEB8A839B8309
:10455000AC83BD831F821E82AC01BD01F7E0CF306A
:10456000DF07D1F088E0FE013896DE0101900D9260
:104570008A95E1F7198618864A875B876C877D875D
:104580001F861E862896EACF219708501109CF3F33
:104590008FEFD80719F610C0C1E0C093A406809130
:1045A0001707815080931707811106C00E948B2145
:1045B000C093CC021092CF06DF91CF911F910F9143
:1045C000FF90EF90DF90CF9008958091CC02811101
:1045D00022C0109217070E948B211092CE061092D3
:1045E000CF061092C3061092C206E7EDF6E080E017
:1045F00090E0A0E8BFEB1182108282839383A483B2
:10460000B58317821682389627E0E731F20799F7CB
:1046100081E08093CC0208958091AD0681110C94C5
:10462000E52208950E940C231092AD0668E070E028
:104630008DE093E00C9468271F920F920FB60F92B3
:1046400011244F925F926F927F92AF92BF92CF925E
:10465000DF92EF92FF920F931F932F933F934F930D
:104660005F936F937F938F939F93AF93BF93CF93FA
:10467000DF93EF93FF938091A9069091AA06A091F2
:10468000AB06B091AC060196A11DB11D8093A906A1
:104690009093AA06A093AB06B093AC066091A906CE
:1046A0007091AA068091AB069091AC060E940E2BE9
:1046B0006B017C0120E030E040E85CE36091A506FE
:1046C0007091A6068091A7069091A8060E94222CC0
:1046D0009B01AC01C701B6010E94612A87FD4AC156
:1046E0001092A9061092AA061092AB061092AC0680
:1046F0008091CF06811105C0C091CE06CC2309F46C
:1047000028C10E94361FEC018091CE06811102C0A3
:1047100010E0E7C08091C4069091C5060E94271F53
:104720002091C2063091C3068217930788F38091C7
:10473000C4069091C5060E94271F2091C2063091A1
:10474000C3067C01E21AF30AD093C506C093C406DF
:104750000091C6061091C706C80101969093C7063E
:104760008093C6060E94361F9093D6068093D50686
:10477000A090C906B090CA068091C6069091C7065F
:104780008A159B0560F0C091C806CC2329F01092D1
:10479000C7061092C60603C00E94E522DAC08091C7
:1047A000CD06C091C606D091C706C090CB06D0906A
:1047B000CC06811131C0F80153E0EE0FFF1F5A956E
:1047C000E1F7EC0DFD1DDE0163E0AA0FBB1F6A954A
:1047D000E1F7AC0DBD1D2D913D914D915C91608136
:1047E0007181828193810E94612A811115C081E0CB
:1047F0008093CD064FE050E060E070E0CB010E9476
:1048000096211093C7060093C6068FE090E0909320
:10481000C3068093C20664C01092CD068E0133E0B9
:10482000000F111F3A95E1F70C0D1D1DF801648171
:104830007581868197810E94DF2A9B01A0E6BAEEEE
:104840000E94E52920E03EE140E050E00E94C329BB
:10485000F1E0AF1AB108412C4EE1542E612C712CBD
:104860002E153F0550F0D093C706C093C606E2163A
:10487000F306E0F0C1E0D0E01CC0085F1F4FCA158E
:10488000DB0588F7E21AF30A2196F8016481758145
:10489000868197810E94DF2A9B01A0E6BAEE0E94E2
:1048A000E529A30192010E94C329DACFE901CE19BB
:1048B000DF098091C6069091C70623E0880F991FF3
:1048C0002A95E1F7F601E80FF91F60817181828175
:1048D0009381AE010E949621D093C306C093C20675
:1048E00011E08091CF06882361F18091D206811179
:1048F00003C08091D306811111E0C7EDD6E0E12C11
:10490000F12C8091170790E0E816F906D4F48E8117
:104910009F8101978E3F9F4F78F4888199810E94F3
:10492000271F2E813F818217930730F06A817B8198
:104930008C819D810E946A222FEFE21AF20A28964A
:10494000E0CFC091A406CC2319F01092A40601C0B8
:10495000C12F8091CF06811107C08091CE068111B1
:1049600003C00E948B2106C0CC2321F00E94F724B3
:104970000E94321EFF91EF91DF91CF91BF91AF91D5
:104980009F918F917F916F915F914F913F912F9167
:104990001F910F91FF90EF90DF90CF90BF90AF905D
:1049A0007F906F905F904F900F900FBE0F901F9071
:1049B00018950F931F938091180790911907A09154
:1049C0001A07B0911B078C019D010871112722273E
:1049D0003327BC01CD01083111052105310511F442
:1049E000606201C06F7D1F910F910C942A158F9208
:1049F0009F92AF92BF92CF92DF92EF92FF920F936E
:104A00001F93CF93DF93E0911707EE2309F447C27A
:104A1000E15048E0E402F0011124E952F94F02812B
:104A20001381D481C58120E030E0A901B8018D2F28
:104A30009C2F0E94612A18160CF031C28091D50675
:104A40009091D6060E94271F7C0164E670E00E94C8
:104A5000222EE091D4068E2F90E08930910508F047
:104A6000D3C1FC01E459FF4F0C944A2E1092D30697
:104A7000CBC11092D30681E08093D206C5C11092BB
:104A8000D3066431710530F46A30710508F422C12F
:104A900089E105C0693C710508F01CC188E180937B
:104AA0008D03B2C11092D30620E030E040EA52E418
:104AB000B8018D2F9C2F0E94612A87FDA5C120E09F
:104AC00030E040E253E4B8018D2F9C2F0E94612A10
:104AD00087FF28C00E943F2968E270E00E94362EBE
:104AE000BC01645C7F4F072E000C880B990B0E9461
:104AF000102B8B01D82FC92F5BE0E516F10408F4C9
:104B0000A5C085E1E816F10408F041C12EECA7012B
:104B10002403C001259F900D1124865E9B4F6AE0FF
:104B200070E098C020E030E040EA53E4B8018D2FF7
:104B30009C2F0E94612A87FF26C00E943F2968EEB1
:104B400073E00E94362EBC0168517C4F072E000C8A
:104B5000880B990B0E94102B8B01D82FC92F56E080
:104B6000E516F10408F472C085E1E816F10408F0D6
:104B70000EC12EECA7012403C001259F900D112426
:104B8000865E9B4F65C020E030E040E254E4B8010F
:104B90008D2F9C2F0E94612A87FF28C00E943F29E9
:104BA00060ED77E00E94362EBC016854744F072EEA
:104BB000000C880B990B0E94102B8B01D82FC92F4A
:104BC00050E1E516F10408F441C085E1E816F1046E
:104BD00008F0DDC02EECA7012403C001259F900D35
:104BE0001124865E9B4F65E070E034C020E030E029
:104BF00040EA54E4B8018D2F9C2F0E94612A87FF60
:104C000003C10E943F2960ED77E00E94362EBC016F
:104C10006854744F072E000C880B990B0E94102BC0
:104C20008B01D82FC92F54E2E516F10478F083E305
:104C3000E816F10408F0ABC02EECA7012403C00174
:104C4000259F900D11248A50964F02C082E327CFF2
:104C50006FE070E00E94222E69C081E08093D3064D
:104C60006431710540F46A30710540F520E030E0B0
:104C700040E85EE327C0693C710508F088C080E029
:104C800090E00E940E2B20E030E040EA51E40E94C8
:104C9000F42920E030E044E353E40E94662A9B01BB
:104CA000AC010E94222C20E030E048E451E40E9454
:104CB000222C0E94DF2A8CE0861BF1CE20E030E01F
:104CC00040E05FE3B8018D2F9C2F0E94222C8B01C6
:104CD000D82FC92F8CE0E3CE81E08093D3062AE061
:104CE000269FC001279F900D112468EB7BE00E9456
:104CF000222EBC016C5D754077FF03C071956195F4
:104D000071097727072E000C880B990B0E94102B36
:104D10002EE333EC4EE259E30E94222C20E030E0F7
:104D200040EC5EE30E94F5290E94DF2A60938D0328
:104D30006BC081E08093D306C70183709927892BCC
:104D4000F1F0C7018170992724E6289FB001299FBF
:104D5000700D112480E090E00E940E2B20E030E0E6
:104D600040E05EE30E94222C20E030E040E45FE37C
:104D70000E94F5290E94DF2A60938D0303C082E31D
:104D800080938D0357E0E522FF24EF28E9F5109288
:104D90008D033AC081E08093D30682E380938D0334
:104DA0006739710588F180E090E00E940E2B20E0C9
:104DB00030E047E153E40E94F42920E030E04AE784
:104DC00054E40E94662A20E030E048E452E40E9465
:104DD000222C20E030E040EA51E40E94562B0E9451
:104DE000D82A660F771F660F771FFB01EE57FA4F21
:104DF0002081318142815381B8018D2F9C2F0E94E7
:104E0000222C8B01D82FC92F8091D206882309F438
:104E10004BC00E94361FBC0180E090E00E940E2B28
:104E200020E030E048E451E40E94662A20E030E0CF
:104E300040EA51E40E94562B6B017C0120E030E0F7
:104E4000A9010E94612A87FF09C020E030E040EA02
:104E500051E4B601C7010E94F52902C0B601C7019D
:104E60004B015C01C501B4010E94D82A660F771F6F
:104E7000660F771FFB01EE57FA4F608171818281C7
:104E8000938120E030E040E05FE30E948F2C9B01A3
:104E9000AC01B8018D2F9C2F0E94222C08C060E02D
:104EA00070E080E090E003C0B8018D2F9C2F6B0173
:104EB0007C01C701B601DF91CF911F910F91FF9047
:104EC000EF90DF90CF90BF90AF909F908F9008951C
:104ED000CF92DF92EF92FF92CF93DF932091D10692
:104EE00020FD08C0DF91CF91FF90EF90DF90CF9031
:104EF0000C94E5227B01EC018091D006811102C067
:104F00000E94511B8091CF0681110E94E52281E011
:104F10008093CE061092CD06D093CC06C093CB06DC
:104F2000F092CA06E092C9061092C8061092C7060F
:104F30001092C6066C817D818E819F810E94DF2A3E
:104F40009B01A0E6BAEE0E94E529C12C2EE1D22EEB
:104F5000E12CF12CA70196010E94C3296881798177
:104F60008A819B81A9010E9496210E94361F9093FD
:104F7000C5068093C4068091CB069091CC06E09143
:104F8000C606F091C70633E0EE0FFF1F3A95E1F732
:104F9000E80FF91F64817581868197810E94DF2A5D
:104FA0009B01A0E6BAEE0E94E529A70196010E94A6
:104FB000C3293093C3062093C206DF91CF91FF909F
:104FC000EF90DF90CF900895EF92FF920F931F9391
:104FD000CF93DF937C018B010E945E12811119C077
:104FE000E70101151105A1F08091E80085FD0AC0D7
:104FF0008091E8008E778093E8000E945E128823FB
:1050000081F307C089918093F10001501109E9CF24
:1050100080E0DF91CF911F910F91FF90EF90089565
:105020001F93CF93DF93CDB7DEB767970FB6F89492
:10503000DEBF0FBECDBF4B8B5C8B6D8B7E8B8F8BA2
:1050400061111092620686E09E01235F3F4FD901F5
:10505000E82F1D92EA95E9F795E0FE017396D901D4
:1050600001900D929A95E1F79C894E895F897B8921
:105070007D879E876F87598B488BF901DE011796D4
:1050800001900D928A95E1F7CE0107960E943213A6
:1050900081113EC086E0FE013796DE011196019037
:1050A0000D928A95E1F7FF81E8856A857B85611518
:1050B000710531F0EF3F31F481E0FF3F19F403C097
:1050C00081E001C080E080FD23C02091270630E010
:1050D000C9010196877099274091580650E08417BE
:1050E000950779F1F983EA837D836C8396E0929F3B
:1050F000D001939FB00D1124A85DB94FFE013196E8
:1051000001900D929A95E1F7809327060E94B21ABA
:1051100016E080915806909127068917F9F0189F9C
:10512000C0011124885D994F0E9432138823B1F089
:105130008091580690E001968770992780935806D1
:10514000E8CF0E9484151092270610925806E1E2DB
:10515000F6E086E0DF011D928A95E9F767960FB6C3
:10516000F894DEBF0FBECDBFDF91CF911F910895A0
:105170008295982F937344E0949F900111248C7C26
:1051800086958695282B822F8575880F2A7A2695F5
:10519000822B0895CF92DF92EF92FF92CF93C82F88
:1051A00020E8829FC001112460E170E082579C4F8B
:1051B0000E946827C12CD12C7601C39404C0CC0C6A
:1051C000DD1CEE1CFF1CCA95D2F76C2D83E090E02D
:1051D0000E945D29C701B601CF91FF90EF90DF904B
:1051E000CF900C947A158F929F92AF92BF92CF92EC
:1051F000DF92EF92FF92CF93DF93EC016881798188
:105200008A819B81611571058105910521F464E214
:1052100079ED8BE597E02DE133EF41E050E00E941E
:10522000912949015A019B01AC01A7EAB1E40E940E
:10523000B0296B017C01ACEEB4EFA50194010E9492
:10524000BE29DC01CB018C0D9D1DAE1DBF1DB7FF1E
:1052500003C00197A109B04888839983AA83BB83BF
:105260009F77DF91CF91FF90EF90DF90CF90BF902D
:10527000AF909F908F9008950E94F328089580E04A
:1052800091E00E94F3280895A0E0B0E0809300012F
:1052900090930101A0930201B09303010895F9993D
:1052A000FECF92BD81BDF89A992780B50895A8E1F7
:1052B000B0E042E050E00C948329262FF999FECF0C
:1052C00092BD81BDF89A019700B4021639F01FBA59
:1052D00020BD0FB6F894FA9AF99A0FBE0895039676
:1052E000272F0E945E290E945D29252F0E945E299A
:1052F000242F0C945E290196272F0E945E290C947E
:105300005D29DC01CB01FC01F999FECF06C0F2BD9D
:10531000E1BDF89A319600B40D9241505040B8F773
:105320000895052E97FB1EF400940E94A82957FDAE
:1053300007D00E94C32907FC03D04EF40C94A8297F
:1053400050954095309521953F4F4F4F5F4F0895B1
:1053500090958095709561957F4F8F4F9F4F0895E1
:105360000E94E529A59F900DB49F900DA49F800DEC
:10537000911D11240895B7FF0C94B0290E94B02903
:10538000821B930B0895A1E21A2EAA1BBB1BFD01E1
:105390000DC0AA1FBB1FEE1FFF1FA217B307E40714
:1053A000F50720F0A21BB30BE40BF50B661F771F6C
:1053B000881F991F1A9469F760957095809590954C
:1053C0009B01AC01BD01CF010895A29FB001B39F25
:1053D000C001A39F700D811D1124911DB29F700DFE
:1053E000811D1124911D08955058BB27AA270E94A2
:1053F0000C2A0C94E82B0E94DA2B38F00E94E12B47
:1054000020F039F49F3F19F426F40C94D72B0EF4B6
:10541000E095E7FB0C94C32BE92F0E94F92B58F37E
:10542000BA17620773078407950720F079F4A6F589
:105430000C941B2C0EF4E0950B2EBA2FA02D0B0113
:10544000B90190010C01CA01A0011124FF27591BC9
:1054500099F0593F50F4503E68F11A16F040A22FCF
:10546000232F342F4427585FF3CF46953795279540
:10547000A795F0405395C9F77EF41F16BA0B620B3F
:10548000730B840BBAF09150A1F0FF0FBB1F661F86
:10549000771F881FC2F70EC0BA0F621F731F841FC9
:1054A00048F4879577956795B795F7959E3F08F0EF
:1054B000B0CF9395880F08F09927EE0F97958795B1
:1054C00008950E949F2B08F481E008950E947A2A93
:1054D0000C94E82B0E94E12B58F00E94DA2B40F04C
:1054E00029F45F3F29F00C94C32B51110C941C2C10
:1054F0000C94D72B0E94F92B68F39923B1F3552311
:1055000091F3951B550BBB27AA27621773078407D6
:1055100038F09F5F5F4F220F331F441FAA1FA9F36C
:1055200035D00E2E3AF0E0E832D091505040E6955A
:10553000001CCAF72BD0FE2F29D0660F771F881FBB
:10554000BB1F261737074807AB07B0E809F0BB0BAE
:10555000802DBF01FF2793585F4F3AF09E3F5105C2
:1055600078F00C94C32B0C941C2C5F3FE4F3983E12
:10557000D4F3869577956795B795F7959F5FC9F7AB
:10558000880F911D9695879597F90895E1E0660F2C
:10559000771F881FBB1F621773078407BA0720F0A5
:1055A000621B730B840BBA0BEE1F88F7E09508950E
:1055B0000E94DF2A6894B1110C941C2C08950E945B
:1055C000012C88F09F5798F0B92F9927B751B0F068
:1055D000E1F0660F771F881F991F1AF0BA95C9F777
:1055E00014C0B13091F00E941B2CB1E008950C94CE
:1055F0001B2C672F782F8827B85F39F0B93FCCF381
:10560000869577956795B395D9F73EF490958095F3
:10561000709561957F4F8F4F9F4F0895E89409C013
:1056200097FB3EF490958095709561957F4F8F4FD5
:105630009F4F9923A9F0F92F96E9BB279395F695EB
:10564000879577956795B795F111F8CFFAF4BB0F69
:1056500011F460FF1BC06F5F7F4F8F4F9F4F16C0CD
:10566000882311F096E911C0772321F09EE8872F57
:10567000762F05C0662371F096E8862F70E060E013
:105680002AF09A95660F771F881FDAF7880F96958C
:10569000879597F908950E94DA2B20F019F00E945F
:1056A000E12B50F40C94D72B0C941C2CE92F0E9466
:1056B000F92B88F35523B1F3E7FB621773078407CF
:1056C0009507A8F189F3E92FFF2788232AF031975E
:1056D000660F771F881FDAF7952F5527442332F07E
:1056E00091505040220F331F441FD2F7BB27E91BB4
:1056F000F50B621B730B840BB109B1F222F4620F3C
:10570000731F841FB11D31972AF0660F771F881F02
:10571000BB1FEFCF9150504062F041F0882332F030
:10572000660F771F881F91505040C1F793950C94D6
:10573000C92B8695779567959F5FD9F7F7CF990F16
:105740000008550FAA0BE0E8FEEF16161706E8074B
:10575000F907C0F012161306E407F50798F0621B6C
:10576000730B840B950B39F40A2661F0232B242B41
:10577000252B21F408950A2609F4A140A6958FEF60
:10578000811D811D089597F99F6780E870E060E0B2
:1057900008959F3F31F0915020F487957795679554
:1057A000B795880F911D9695879597F908959FEF66
:1057B00080EC089500240A941616170618060906A8
:1057C000089500240A941216130614060506089577
:1057D000092E0394000C11F4882352F0BB0F40F4FF
:1057E000BF2B11F460FF04C06F5F7F4F8F4F9F4F3F
:1057F000089557FD9058440F551F59F05F3F71F0C1
:105800004795880F97FB991F61F09F3F79F0879527
:105810000895121613061406551FF2CF4695F1DFB0
:1058200008C0161617061806991FF1CF8695710540
:10583000610508940895E894BB2766277727CB0174
:1058400097F908950E94352C0C94E82B0E94DA2BCE
:1058500038F00E94E12B20F0952311F00C94C32B1B
:105860000C94D72B11240C941C2C0E94F92B70F350
:10587000959FC1F3950F50E0551F629FF001729FF5
:10588000BB27F00DB11D639FAA27F00DB11DAA1F04
:10589000649F6627B00DA11D661F829F2227B00D51
:1058A000A11D621F739FB00DA11D621F839FA00DDC
:1058B000611D221F749F3327A00D611D231F849F2C
:1058C000600D211D822F762F6A2F11249F57504083
:1058D0009AF0F1F088234AF0EE0FFF1FBB1F661FFE
:1058E000771F881F91505040A9F79E3F510580F0C7
:1058F0000C94C32B0C941C2C5F3FE4F3983ED4F320
:10590000869577956795B795F795E7959F5FC1F76A
:10591000FE2B880F911D9695879597F90895FA01AA
:10592000EE0FFF1F309621053105A1F161157105BC
:1059300061F48038BFE39B0749F168949038810592
:1059400061F08038BFEF9B0741F099234AF5FF3F94
:10595000E1053105210519F1E8940894E795D9018D
:10596000AA2329F4AB2FBE2FF85FD0F310C0FF5F3E
:1059700070F4A695E0F7F73950F019F0FF3A38F4D3
:105980009F779F930DD00F9007FC9058089546F095
:105990000C94D72B60E070E080E89FE308954FE718
:1059A0009F775F934F933F932F930E948A2D2F9160
:1059B0003F914F915F910E94222C0C94E72C29F487
:1059C00016F00C94C32B0C941B2C0C94D72B0E9418
:1059D000012CA8F39638A0F707F80F92E8942BE370
:1059E0003AEA48EB5FE70E94382C0F920F920F9231
:1059F0004DB75EB70F920E94D22DEAEEF0E00E9402
:105A0000192D4F915F91EF91FF91E595EE1FFF1FCB
:105A100049F0FE57E0684427EE0F441FFA95E1F77E
:105A20004195550B0E944C2D0F9007FE0C94402D74
:105A30000895DF93CF931F930F93FF92EF92DF921E
:105A40007B018C01689406C0DA2EEF010E94352C90
:105A5000FE01E894A5912591359145915591A6F3C4
:105A6000EF010E940C2AFE019701A801DA9469F760
:105A7000DF90EF90FF900F911F91CF91DF910895EC
:105A80009B01AC0160E070E080E89FE30C94662A23
:105A90000C94C32B0C94C92B0E94012CD8F399238E
:105AA000C9F3940F511DA3F39150504094F059F055
:105AB000882332F0660F771F881F91505040C1F73E
:105AC0009E3F51052CF7880F911D9695879597F964
:105AD00008955F3FACF0983E9CF0BB278695779584
:105AE0006795B79508F4B1609395C1F7BB0F58F768
:105AF00011F460FFE8CF6F5F7F4F8F4F9F4FE3CF71
:105B00000C941C2C16F00C94C92B0C94D72B689475
:105B10000C94C32B0E94012CA8F39923C1F3AEF37C
:105B2000DF93CF931F930F93FF92C92FDD27882315
:105B30002AF02197660F771F881FDAF720E030E000
:105B400040E85FEB9FE3883920F0803E38F02196F3
:105B50008F770E94F529E2E1F1E004C00E94F52967
:105B6000EFE3F1E00E94192D8B01BE01EC01FB2E49
:105B70006F5771097595771F880B990B0E94102B31
:105B800028E132E741E35FE30E94352CAF2D980115
:105B9000AE01FF900F911F91CF91DF910E940C2ACF
:105BA0000C94E82BFA01DC01AA0FBB1F9B01AC018E
:105BB000BF5728F4222733274427507820C0B751F5
:105BC00090F4AB2F0024469537952795011CA3959B
:105BD000D2F3002071F0220F331F441FB395DAF384
:105BE0000ED00C94F42961307105A0E88A07B946FB
:105BF00030F49B01AC016627772788279078309690
:105C000021F020833183428353830895DB018F93F6
:105C10009F930E94B029BF91AF91A29F800D911DCB
:105C2000A39F900DB29F900D11240895991B79E0C8
:105C300004C0991F961708F0961B881F7A95C9F71C
:105C400080950895AA1BBB1B51E107C0AA1FBB1F6B
:105C5000A617B70710F0A61BB70B881F991F5A95F8
:105C6000A9F780959095BC01CD01089597FB072E6B
:105C700016F4009407D077FD09D00E94222E07FC6D
:105C800005D03EF4909581959F4F0895709561954C
:105C90007F4F0895EE0FFF1F0590F491E02D0994BA
:105CA000FB01DC0104C08D910190801921F4415069
:0E5CB0005040C8F7881B990B0895F894FFCF59
:105CBE000100000000005C44000080415C978A44B3
:105CCE000000804152D0A444000080410000DC441A
:105CDE00000080410000DC44000000410AA7CF44D0
:105CEE00000000415CFFB8440000004152D0A444C3
:105CFE00000000411FD59244000000415C978A4489
:105D0E000000004148F176440000004100005C4470
:105D1E000000004100005C44000080411F156944F2
:105D2E000000804148F176440000804100D082445A
:105D3E00000080415C978A4400008041A4D0244436
:105D4E000000804100005C44000080411FD5924459
:105D5E00000080415CFFC344000080410000000051
:105D6E00000000005CFF4344000080411FD59244B8
:105D7E00000080410000DC440000804152D02445E8
:105D8E0000008041000000000000000000005C44A4
:105D9E000000804148F17644000080415C978A44BF
:105DAE00000080411FD592440000804152D0A4448F
:105DBE00000080410300005C440000004100005CD4
:105DCE00440000004100005C440000004100005C03
:105DDE00440000004148F176440000C04000005CE1
:105DEE00440000C04048F176440000C04000005C12
:105DFE00440000C04048F176440000C04000005C02
:105E0E00440000C04048F176440000C04000005CF1
:105E1E00440000C04052D02445000000410000DC88
:105E2E00440000004152D0A44400004041012F1E06
:105E3E00861E2E1E9D0D990D350D640048F176447B
:105E4E000000A041F6F0F6440000004152909B4441
:105E5E000000A041F6F0F6440000004100005C4452
:105E6E00000000410000DC44000000410000DC4462
:105E7E000000004100005C44000000410100005C95
:105E8E00440000004148F17644000000415C978ACE
:105E9E0044000000411FD592440000004152D0A49E
:105EAE0044000000415CFFB844000000410AA7CF47
:105EBE0044000000410000DC44000000410000DC12
:105ECE0044000000410AA7CF44000000415CFFB827
:105EDE00440000004152D0A444000000411FD5925E
:105EEE0044000000415C978A440000004148F1766E
:105EFE00440000004100005C440000004100005CD2
:105F0E00440000004148F17644000000415C978A4D
:105F1E0044000000411FD592440000004152D0A41D
:105F2E0044000000415CFFB844000000410AA7CFC6
:105F3E0044000000410000DC4400000041320AA78A
:105F4E00CF44000000410000DC440000004100008E
:105F5E0000000000804052D0244500008041000027
:105F6E000000000000000000000000000000000023
:105F7E000000000000000000000000000000000013
:105F8E000000000000000000000000000000000003
:105F9E0000000000000000000000000000000000F3
:105FAE0000000000000000000000000000000000E3
:105FBE0000000000000000000000000000000AA722
:105FCE00CF44000000410000DC440000004100000E
:105FDE0000000000804052D02445000040410000E7
:105FEE000000000080400AA74F450000404100001D
:105FFE000000000000000000000000000000000093
:10600E000000000000000000000000000000000082
:10601E000000000000000000000000000000000072
:10602E000000000000000000000000000000000062
:10603E0000000000000000000000000000000AA7A1
:10604E00CF44000000410000DC440000004100008D
:10605E0000000000804052D02445000000410000A6
:10606E000000000080405CFF384500000041000049
:10607E0000000000804052D0244500000041000086
:10608E000000000000000000000000000000000002
:10609E0000000000000000000000000000000000F2
:1060AE0000000000000000000000000000000000E2
:1060BE0000000000000000000000000000000002D0
:1060CE00040507090B0C0E1011131517181A1C1DB9
:1060DE001F2123242628292B2D2F303234353739F2
:1060EE003B4032224E021C02FA01B402CD02E602FD
:1060FE00818283E200E900EA00B500B600B700CD68
:10610E00008301CC008A0192019401210223022412
:10611E00022502260227022A02B300B4006F007085
:10612E00009295353693F1F03067F4F5F6F79496C4
:10613E0034973149803F5D8B803FF8BF803FCAE185
:10614E00803F73ED803FCAE1803FF8BF803F5D8B9B
:10615E00803F3149803F0000803FF16D7F3F75EAFF
:10616E007E3F4C827E3F833F7E3F84287E3F833F2F
:10617E007E3F4C827E3F75EA7E3FF16D7F3F000091
:02618E00803F50
:00000001FF
